:03000000020100FA
:03000B00020916D1
:100100007880E4F6D8FD7B6474E1D1EADBFA758986
:1001100001759240D2A9D2AFD28C12092C120B33A6
:100120003000FDC2003000FDC2003000FDC20012F0
:100130000A35F1943149300202912AD1F03000F4AD
:10014000C20080F0C28FC28E222094FC758B007595
:100150008D00758911D28E208FEA3094FAC28E8577
:100160008B28858D29758B00758D00D28EE529B47D
:10017000000CE528B49603020C5A40C880F9B4017B
:1001800013E528B4F0030205C9B430030205C940E1
:10019000E60205C9B40203020523B4030302067E86
:1001A000B40903020472B40A03020472B40D030218
:1001B0000281B40E03020281B40C0DE528B4800361
:1001C000D2022240FB020281B41003020211B411D8
:1001D0000280F8B4120280F3B4130280EEB41E035E
:1001E000020B72B41F0280F8B4200280F3B4210223
:1001F00080EEB4220302035AB4230302035AB42448
:10020000BF02035A0205230205C9C28FC28ED20261
:1002100022208FF62094FAC28E752400858B2885C3
:100220008D29758B00758D00D28EE529B4100302DF
:100230000241B41103020241B41203020241B41399
:10024000C97B3074E1D1EADBFAE522B40905D1605B
:1002500002025F752300752209120AF4120A827BDA
:100260000174E1D1EADBFA714722C28FC28E3028D5
:1002700005C228D20222D2287B3C74E1D1EADBFA03
:1002800022208FE62094FAC28E752400858B288563
:100290008D29758B00758D00D28EE529B406CB7F34
:1002A000307E007D007C007B007A0079003094FD78
:1002B000C28EE58D858B28758B00758D00D28EB42E
:1002C00002030202D2B401A2E528B47C030202D2E6
:1002D0004098208F952094FAC28EE58D858B2875E5
:1002E0008B00758D00D28EB402030202FAB4010EA7
:1002F000E528B440030202FA40D6C30202FFD3EE5F
:1003000013FEED13FDEC13FCEB13FBEA13FAE913F8
:10031000F9DF9A892A8A2B8B2C8C2D8D2E8E2F8D8E
:10032000407541008C26E522B40405D16002033CEF
:10033000752300752204120AF41209DB7B2D74E187
:10034000D1EADBFA714722C202752500C203C28ED0
:10035000C28F22C28FC28ED20222208FF62094FA40
:10036000C28E752400858B28858D29758B00758D2F
:1003700000D28EE529B4100302039AB411030203DC
:100380009AB4120302039AE529B40703020392B454
:1003900008C1E522B403BC02041F7F207D007C005D
:1003A0007B007A003094FDC28EE58DB402A5758B7A
:1003B00000758D00D28E208F9A2094FAC28EE58D22
:1003C000858B28758B00758D00D28EB402050203D3
:1003D000E08080B4010EE528B490030203E040F110
:1003E000C30203EAB4000280E8D3ED13FDEC13FC72
:1003F000EB13FBEA13FADFAC8A2A8B2B8C2C8D2DA6
:100400008A268C40754100E522B40305D1600204C0
:100410001F752203752300120AF41209AAF1947BB6
:100420001E74E1D1EADBFA714722C28EC28FC2028A
:10043000752500752300752208120AF4120AB97B8B
:10044000FA74E1D1EADBFA22C28EC28F3000F9C21F
:1004500000C203C2293000F922C28F302905C22907
:10046000D20222D229C28F7B1474E1D1EADBFAC214
:100470000322208FE42094FAC28E752400858B28F5
:10048000858D29758B00758D00E529B40203020462
:100490009EB401C5E528B4900302049E40BB7F18BA
:1004A0007D007C007B00D28E3094FDC28EE58DB441
:1004B0000204C30204BCB4000280F7D3ED13FDECC8
:1004C00013FCEB13FB748CD1EA758B00758D00DF88
:1004D000D5C2298B2A8C2B8D2CEB547FF54075418E
:1004E00000EC540FF526EB20E704C30204EFD3E53C
:1004F0002633F526E522B4050E753B20753C2075A4
:100500003D20D160020513752205752300120AF4FF
:100510001209EF71477B0374E1D1EADBFA22D202C0
:10052000C20322208FF82094FAC28E752400858B96
:1005300028858D29E529B4090302053FB40ADF7433
:100540003CD1EA2094D83094FD74C0D1EA7E007F7B
:10055000097D007C00E5905410FE7480D1EAE5909E
:100560005410C39E60B8ED13FDEC13FC7480D1EA07
:10057000DFE3200313ECB400A7EDB400A3D2037FA4
:100580000F74FFD1EADFFA22C203ECF45480FCF5C9
:1005900040EDF4FDF5417F07C3ED13FDEC13FCDFE7
:1005A000F88C2A8D2BE522B40705D1600205BB75B6
:1005B0002207752300120AF4120A9C71477BC87443
:1005C000E1D1EADBFA22D202227F0F7D007C0020FB
:1005D0008FF42094FA752400C28E858B28858D298E
:1005E000758B00758D00D28EE529B4070BE528B414
:1005F0006C0280D2401880CE4005020C7380C7B4D4
:10060000020302060A40F602060EC302060FD3C218
:100610008EEC33FCED33FD7432D1EA3094FD758BF2
:1006200000758D00D28E2094FDDFA48C2A8D2BEDD9
:100630000303541FF526852A40E52B5403F541E5B5
:1006400022B40605D16002065575230075220612F4
:100650000AF4120A0371477B2574E1D1EADBFA221E
:10066000E523B4010412089822B402041208CC2233
:10067000B403031207C922D202C2032280F97E000A
:100680007F0C7D007C007524002094FD746ED1EAFF
:1006900074DCD1EAE5905410FE74DCD1EAE59054A4
:1006A00010C39E60D7EC33FCED33FD74D7D1EADF85
:1006B000E38C2A8D2B7F02EC33FCED33FDDFF8EC6D
:1006C0000303F540ED541FF526E522B40105D16082
:1006D0000206DF752201752300120AF41209B871AF
:1006E000477B0A74E1D1EADBFA220000D5E0FB2265
:1006F000309703C201227464D1EA2097F82001F5F3
:10070000D201E522B40015120A17F1943000FDC29F
:10071000003000FDC200120A35F19422E5232401C5
:10072000F523B404537523007400120AF4E522B4CF
:1007300001041209B822B4020412099322B4030678
:100740001209AAF19422B404061209DBF19422B42E
:1007500005041209EF22B40604120A0322B40704A6
:10076000120A9C22B40A04120D2222B40904120AAD
:100770008222120AB9F19422B40107120B15120851
:100780009822B40207120AD31208CC221209C61208
:1007900007C92222C29075800212095F1209677987
:1007A000308780D29012095F12096709B938F2C206
:1007B000907580C012095F1209678780D290120974
:1007C0005F12096709B940F222E522B40805020860
:1007D000A3E522B40426E52F540F120A5CF535E593
:1007E0002FC4540F120A5CF534E52E540F120A5C24
:1007F000F537E52EC4540F120A5CF536E522B40431
:1008000003020807B40313E52D540F120A5CF539EF
:10081000E52DC4540F120A5CF538E522B404030236
:100820000833B40303020833B40523E52CB40003F2
:1008300002084EE52C540F120A5CF53BE522B40584
:100840000302084EE52CC4540F120A5CF53AE52A5F
:10085000540F120A5CF53FE52AC4540F120A5CF5E6
:100860003EE52B540F120A5CF53DE522B40103026C
:100870000894E522B4050BE52BC4540FB400030221
:100880000894E522B40203020894E52BC4540F1225
:100890000A5CF53C12079422E522B407030208A380
:1008A000B4080A753E2D753F2D12079422E5265493
:1008B0000F120A5CF53FE522B4020574200208C855
:1008C000E526C4540F120A5CF53E80DDE522B4082B
:1008D000030208A3E540540F120A5CF53FE540C44B
:1008E000540F120A5CF53EE522B40A03020912B461
:1008F00006030208F7401BE541540F120A5CF53D60
:10090000E522B40603020912E541C4540F120A5C41
:10091000F53C12079422C0D0C0E0E5212401B410B8
:10092000047400D200F521D0E0D0D032758030754B
:1009300090F8315375803031537580303153758064
:100940003C3153758008315375800C3153758006E6
:100950003153227FFF0000000000000000DFF6D2CC
:1009600091000000C29122C0E0C0F04380FFC2901D
:10097000D292C29100D29100E580F5F0C29100D2EE
:100980009100E58045F0C29100C292D0F020E7D9F5
:10099000D0E02278397652087645087643087653B7
:1009A000087638087630120794227839764E087621
:1009B0004508764312079422783976520876430820
:1009C0007635120794227830764308764F087644BD
:1009D00008763A08762008B840FA227839764A082C
:1009E000764108765008764108764E1207942278B0
:1009F00039765308764908765208764308765312BA
:100A00000794227839764408764508764E08764F62
:100A100008764E120794227830764E08764F087684
:100A200020087644087641087654087641087620F6
:100A300008B840FA22783076570876410876490897
:100A4000765408764908764E08764708762E08765A
:100A50002E08762E08762008B840FA22B40A0374CD
:100A60004122401BB40B03744222B40C0374432292
:100A7000B40D03744422B40E037445227446224418
:100A800030227838765308764108764D0876530838
:100A9000765508764E087647120794227838764DB8
:100AA00008764F08765408764F08765208764F0835
:100AB000764C087641120794227839765508764E9E
:100AC00008764B08764E08764F08765708764E1211
:100AD0000794227830764308764F08764D08764D95
:100AE00008764108764E08764408763A087620085B
:100AF000B83EFA227830764608764F087652087665
:100B00004D08764108765408763A08762008B840B1
:100B1000FA12079422783076410876440876520813
:100B2000764508765308765308763A08762008B852
:100B30003EFA227830764308764F087644087645A8
:100B400008762008764108764E08764108764C08EB
:100B50007659087653087645087652087620087646
:100B60005608763112079422C296D2021203490225
:100B70000D18208FF32094FAC28E752400858B28DF
:100B8000858D29758B00758D00D28EE529B40F03F4
:100B9000020B9CB41003020B9CB411CC7F087D00A7
:100BA0007A02208FC33094FAC28EE58D858B28752A
:100BB0008B00758D00D28EB40203020BCAB401A85B
:100BC000E528B49003020BCA401B208F9B2094FAA7
:100BD000C28EE58D858B28758B00758D00D28EB405
:100BE0000205020BF48081B4010EE528B430030243
:100BF0000BF440F1C3020BF9D3ED13FDDFA4DA02CD
:100C000080248D268D2B7D007F087B0474E11206E5
:100C1000EADBF9208FCF2094FAC28E758B00758D98
:100C200000D28E020BA28D408D2AE522B40A061254
:100C30000660020C4175220A752300120AF4120D97
:100C4000221203477B0A74E11206EADBF92212033F
:100C50004922D202120349020D18208FF12094FA82
:100C6000C28E752400858B28858D29758B00758D26
:100C700000D28EE529B42103020C87400280D3B450
:100C80001B03020C8740CB790A7D007C00208FC2B9
:100C90003094FAC28EE58D858B28758B00758D009A
:100CA000D28EB4010CE528B41803020CBB400C80B2
:100CB000A1E528B49603020CBB4097208F942094A2
:100CC000FAC28EE58D758B00758D00D28EB4180337
:100CD000020CD84003020CDCC3020CDDD3EC33FC65
:100CE000ED33FDD9A8C28E8C2A8D2BEC543FF540F4
:100CF0007F06ED13FDEC13FCDFF85407F526E52223
:100D0000B40206120660020D157522027523001248
:100D10000AF41209931203477B1E74E11206EADB00
:100D2000F9227838764408764108764508765708DF
:090D3000764F08764F1207942259
:00000001FF
